:100B3A0000C000F900A400B000990092008200F8F9
:100B4A00008000900088008300C600A10086008E05
:0A0DBD00E51125E0F511EF421122C7
:0D0D4000E51125E0F511EFF45401421122F8
:040E3500EF52112245
:070DF200EFF454015211223D
:040E3900EF42112251
:070DF900EFF4540142112246
:0E0D1600E511F45401FFE51154FE4FF51122D2
:060E2300E5115401FF225D
:0D0D4D00E511C313FFE51154015FF51122FC
:0D0D5A00E511C313FFE51154014FF51122FF
:070BF200EE1313135401FD83
:0E0BF900E51125E0F511EDF45F5401421122E3
:0E0D2400E51125E0F511EFF45D5401421122B6
:08000300EDF45F5401521122DB
:080DDA00EFF45D5401521122F7
:080DE200EDF45F5401421122FF
:080DEA00EFF45D5401421122F7
:070E0000EDF45F5401FF2235
:070E0700EFF45D5401FF222E
:0D0D6700E51825E0FFE51154014FF51822B5
:0D0D7400E5185401FFE51154FE4FF5112262
:100C0700E5185401FFE51154FE4FF511E518C3131C
:030C1700F51822AB
:100CF7008E5E8F5FE55F2DFFE55E3C8FF002075F3D
:100C1A008E608F61C3E5619DFFE5609C8FF00207DE
:010C2A005F6A
:090DD10012069EEE8FF002075F8E
:0F0D07008B5B8A5C895D1206B0EE8FF002075F8E
:070E0E00E475F00102072763
:070E150074FFF5F00207274E
:100C2B008E628F63E5625CFFE5635DCF8FF0020739
:010C3B005F59
:100C3C008E648F65E5644CFFE5654DCF8FF0020740
:010C4C005F48
:100C4D008E668F67E5666CFFE5676DCF8FF00207E7
:010C5D005F37
:100C5E00EFF4FFEEF4FEEF2401FFE43E8FF0020707
:010C6E005F26
:060E2900EFF45401FF226A
:060E2F00EE8FF002075FE8
:0A0DC700EFF4FFEEF48FF002075F77
:100AE4008B4B8A4C894D1206FCFFAEF0AB4EAA4FDD
:100AF400A9501206FCFDAB4BAA4CA94DE5F08DF0B4
:0F0B040012075FAB4EAA4FA950EE8FF002075FAA
:1007D3008E528F538B548A5589567C037DE81206BB
:1007E300B0EFC454F07B00FAAE52AF537C037DE804
:1007F3001206B08C528D53AE52AF537C007D6412FF
:1008030006B0EFFEE4EE4202AE52AF537C007D64CD
:100813001206B08C528D53AE52AF537C007D0A1238
:1008230006B0EFC4F8540FC868FFEEC454F048FE96
:10083300EFFBEE4202AE52AF537C007D0A1206B0CC
:100843008C528D53E5524AFFE5534BAB54AA55A93D
:0708530056CF8FF002075F92
:1008D9008E578F58E558780CCEA2E713CE13D8F867
:1008E9007E00540FFF7C037DE812069E8E598F5AB5
:1008F900E557FF3395E07E00EF540FFF7C007D64E0
:1009090012069EEF255AF55AEE3559F559E558AEB6
:10091900577804CEA2E713CE13D8F87E00540FFF00
:100929007C007D0A12069EEF255AF55AEE3559F5D7
:1009390059E558540F255AF55AE43559F559855A48
:04094900F002075F52
:100B5A00E51125E0F511C3EF9DEC6480F8EE6480A1
:0B0B6A00984004431101225311FE22A9
:100B7500E51125E0F511D3EF9DEC6480F8EE648076
:0B0B8500985004431101225311FE227E
:100B9000E51125E0F511D3EF9DEC6480F8EE64805B
:0B0BA000984004431101225311FE2273
:100BAB00E51125E0F511C3EF9DEC6480F8EE648050
:0B0BBB00985004431101225311FE2248
:100BC600E51125E0F511EF6D7002EE6C600443113E
:060BD60001225311FE2272
:100BDC00E51125E0F511EFB50508EEB50404431158
:060BEC0001225311FE225C
:100C6F00C3EF9DEC6480F8EE64809850035311FE3F
:010C7F002252
:100C8000D3EF9DEC6480F8EE64809840035311FE2E
:010C90002241
:100C9100D3EF9DEC6480F8EE64809850035311FE0D
:010CA1002230
:100CA200C3EF9DEC6480F8EE64809840035311FE1C
:010CB200221F
:0C0D8100EFB50507EEB504035311FE2288
:0C0D8D00EF6D7002EE6C60035311FE224B
:100CB300C3EF9DEC6480F8EE648098400343110118
:010CC300220E
:100CC400D3EF9DEC6480F8EE6480985003431101E7
:010CD40022FD
:100CD500D3EF9DEC6480F8EE6480984003431101E6
:010CE50022EC
:100CE600C3EF9DEC6480F8EE6480985003431101D5
:010CF60022DB
:0C0D9900EF6D7002EE6C6003431101224C
:0C0DA500EFB50507EEB504034311012271
:070E1C00E4FF0FBF0AFC22F6
:100AB400E4FEC2B4120E1CC2B3120E1CD2B3120E48
:100AC4001CD2B4120E1CE4FDEE25E0FE3094034368
:100AD4000601C2B3120E1CD2B30DBD08EBAF062241
:1004BD000510E510C394054003E4F510E510146034
:1004CD005B1470030205791470030205C5240360E3
:1004DD00030206177C0090000DE0540FFD25E0FF90
:1004ED00EC33FE743A2FF582740B3EF583E493FCE6
:1004FD00740193FD43040890010AE0FFC413131324
:10050D00540130E0057DFF02066DEF131313541FE8
:10051D0020E00302066D53057F02066D90000CE08E
:10052D00FEA3E07804CEA2E713CE13D8F87C0054D6
:10053D000FFD25E0FFEC33FE743A2FF582740B3E70
:10054D00F583E493FC740193FD43040490010BE0E7
:10055D0030E0057DFF02066D90010AE0FFC4540FE7
:10056D0020E00302066D53057F02066D90000CE03E
:10057D00FF3395E07C00EF540FFD25E0FFEC33FEDB
:10058D00743A2FF582740B3EF583E493FC7401935A
:10059D00FD43040290010BE0FFC31330E0057DFF26
:1005AD0002066D90010AE0FFC413540720E0030218
:1005BD00066D53057F02066D90000CE0FEA3E078FA
:1005CD000CCEA2E713CE13D8F87C00540FFD25E016
:1005DD00FFEC33FE743A2FF582740B3EF583E493F2
:1005ED00FC740193FD43040190010BE0FF131354C0
:1005FD003F30E0047DFF806890010AE0FFC41313D3
:10060D00540330E05B53057F805690010BE0F9C435
:10061D001313540175F008A4FBAAF0E9C4131313C6
:10062D00540175F010A4FFE5F04AFAEF4BFBE9C455
:10063D0013540175F004A4FFEA45F0FAEB4FFBE902
:10064D00C4540125E0FFE4334AFEEB4FFFE91313D9
:10065D00135401FBEEEF4BF4FFEEF47410FCAD07F9
:10066D007B10C2B3120E1CEC20E704C2B78002D27D
:10067D00B7120E1CED25E0FDEC33FCD2B3120E1CAF
:10068D00DBE0D2B7120E1CC2B5120E1CD2B5020E93
:01069D001C40
:1002D700E52E70030204BC152E0517E517B40517A4
:1002E700AF30EFC4135401F45401FFC43354E0FF9B
:1002F700E53054DF4FF530E517B40A1CAF30EFC4D3
:10030700135401F45401FFC43354E0FFE53054DFC4
:100317004FF530051DE4F517E4F552E552131313B5
:10032700541F2412F8E6FD7C00E5525407FF7401C0
:100337007E00A807088005C333CE33CED8F9FFEE79
:100347005CFEEF5D4E6043E55225E025E0246EF547
:1003570082E43400F583E0FEA3E0FFE55225E025C3
:10036700E0246CF582E43400F583E0FCA3E0C39F4E
:10037700EC9E5016E55225E025E0246CF582E43426
:1003870000F583E475F0011206E6E55225E025E065
:10039700246EF582E43400F583E0FEA3E0FFE55226
:1003A70025E025E0246CF582E43400F583E0FCA326
:1003B700E0C39FEC9E407AE55225E025E0246CF5EA
:1003C70082E43400FEC3E582946CFFEE9400FE7C69
:1003D700007D021206B07C007D021206B07C007D13
:1003E700081206B0741E2FF8C000E6FFC007E552DA
:1003F70025E025E0246CF582E43400FEC3E5829411
:100407006CFFEE9400FE7C007D021206B07C007D3E
:10041700021206B07C007D081206B0AF057401A871
:1004270007088002C333D8FCFED0E04ED000F68028
:1004370079E55225E025E0246CF582E43400FEC31B
:10044700E582946CFFEE9400FE7C007D021206B0FC
:100457007C007D021206B07C007D081206B0741E77
:100467002FF8C000E6FFC007E55225E025E0246C21
:10047700F582E43400FEC3E582946CFFEE9400FE3F
:100487007C007D021206B07C007D021206B07C0063
:100497007D081206B0AF057401A807088002C333B0
:1004A700D8FCF4FED0E05ED000F60552E552642099
:0604B70060030203222293
:1009FA00E51DB41E19AF30EFC413135401F45401AA
:100A0A00FFC4333354C0FFE53054BF4FF530E51D02
:100A1A00B43C1CAF30EFC413135401F45401FFC4A7
:100A2A00333354C0FFE53054BF4FF530E4F51D228F
:03000B0002094D9A
:10094D00C0E0C0D075D008758CEEAF30EF13131327
:10095D005401F45401FF33333354F8FFE53054F7A9
:10096D004FF530053AE53A30E0020516E53AB40A9E
:10097D0015AF30EFC45401F45401FFC454F0FFE53A
:10098D003054EF4FF530E53AB4141AAF30EFC4548C
:10099D0001F45401FFC454F0FFE53054EF4FF5302E
:0A09AD00052E753A00D0D0D0E032DC
:1009B7007594FF752F05E4F530F53190000CF0A321
:1009C700F090010BE054F7F054EFF054DFF054BF10
:1009D700F0547FF090010AE054F7F054EFF054DF41
:1009E700F054BFF0547FF0A3E054FEF054FDF054F0
:0309F700FBF022F0
:040E3D00752F0922E2
:100A3A00E4FFEF25E025E0246CF582E43400F58339
:100A4A00E4F0A3F00FBF20EAE4FF7F4090002CE41B
:100A5A00F0A3DFFCE4FF741E2FF8E4F60FBF04F6E0
:0D0A6A00E4FF74192FF8E4F60FBF04F62224
:0E0D3200758911D2B4D2B9D2A9D28CD2AF2217
:100A7700AFA0EFC3135455FEEF25E054AA4EFF1362
:100A8700135433FEEF25E025E054CC4EFF54F0FE1F
:100A9700E590540F4EF4F522EF540FF4540FF5235D
:0D0AA700120AB4EFF4F5248528800204BD86
:10085A00E4FF74222FF8E6FE743F2FF8A6060FBFB6
:10086A0006F0E4FF74282FF8E6FE74452FF8A60672
:10087A000FBF06F0E4FF74682FF8E6FE74202FF528
:10088A0082E43401F583EEF00FBF20EAE4FF74EC52
:10089A002FF582E43400F583E0FE74402FF582E4FC
:1008AA003401F583EEF00FBF20E4E4FF741E2FF845
:1008BA00E6FE74362FF8A6060FBF04F0E4FF74199B
:0F08CA002FF8E6FE74322FF8A6060FBF04F022B7
:100B13007551011209B7120A3A120D32120A7712ED
:100B2300000E1202D71209FA12085AE55160EDE4D9
:070B3300F551120E3D80E5B3
:10000E00AF2FEF13135401FF120DBDE51130E007B2
:10001E00E490010CF0A3F0E5225401FFE53F5401FA
:10002E00FD120BF9E51130E00D7B017A01790C7FA1
:10003E00017E00120E2FAF22EFC3135401FFAE3F0D
:10004E00EEC3120BF5E51130E00D7B017A01790C50
:10005E007F027E00120E2FAF22EF13135401FFAE5C
:10006E003FEE120BF4E51130E00D7B017A01790CB5
:10007E007F037E00120E2FAF22EF1313135401FFD6
:10008E00AE3F120BF2E51130E00D7B017A01790CD7
:10009E007F047E00120E2FAF22EFC45401FFAE3F3D
:1000AE00EEC45401FD120BF9E51130E00D7B017A1F
:1000BE0001790C7F057E00120E2FAF22EFC4135470
:1000CE0001FFAE3FEEC4120BF5E51130E00D7B01E2
:1000DE007A01790C7F067E00120E2FAF22EFC41329
:1000EE00135401FFAE3FEEC4120BF4E51130E00DD8
:1000FE007B017A01790C7F077E00120E2FAF22EF63
:10010E00C41313135401FFAE3FEEC4120BF3E511EB
:10011E0030E00D7B017A01790C7F087E00120E2FE4
:10012E00E5235401FFE5405401FD120BF9E51130B2
:10013E00E00D7B017A01790C7F097E00120E2FAF44
:10014E0023EFC3135401FFAE40EEC3120BF5E511BE
:10015E0030E00D7B017A01790C7F0A7E00120E2FA2
:10016E00AF23EF13135401FFAE40EE120BF4E51163
:10017E0030E00D7B017A01790C7F0B7E00120E2F81
:10018E00AF23EF1313135401FFAE40120BF2E51120
:10019E0030E00D7B017A01790C7F0C7E00120E2F60
:1001AE00E5245401FFE5415401FD120BF9E5113030
:1001BE00E00D7B017A01790C7F0D7E00120E2FAFC0
:1001CE0024EFC3135401FFAE41EEC3120BF5E5113C
:1001DE0030E00D7B017A01790C7F0E7E00120E2F1E
:1001EE00AF24EF13135401FFAE41EE120BF4E511E1
:1001FE0030E00D7B017A01790C7F0F7E00120E2FFD
:10020E00AF24EF1313135401FFAE41120BF2E5119D
:10021E0030E00D7B017A01790C7F107E00120E2FDB
:10022E00AF24EFC45401FFAE41EEC45401FD120BD6
:10023E00F9E51130E00D7B017A01790C7F117E001A
:10024E00120E2FAF24EFC4135401FFAE41EEC412B1
:02025E000BF59E
:10026000E51130E00D7B017A01790C7F127E0012DE
:100270000E2FAF24EFC413135401FFAE41EEC4128E
:100280000BF4E51130E00D7B017A01790C7F137ED0
:1002900000120E2FAF24EFC41313135401FFAE410D
:1002A000EEC4120BF3E51130E00D7B017A01790CFD
:1002B0007F147E00120E2FE52F5401FF120DBDE5B5
:1002C0001130E01190010CE0FEA3E0FF7B017A0009
:0702D000790C1207D3002294
:03000000020DB13D
:0C0DB100787FE4F6D8FD758187020B13F3
:10069E00EF8DF0A4A8F0CF8CF0A428CE8DF0A42E70
:0206AE00FE222A
:1006B000C2D5EC30E709B2D5E4C39DFDE49CFCEE65
:1006C00030E715B2D5E4C39FFFE49EFE12077EC358
:1006D000E49DFDE49CFC800312077E30D507C3E453
:0606E0009FFFE49EFE22D4
:1006E600C5F0F8A3E028F0C5F0F8E582158270029F
:0606F6001583E038F0223C
:1006FC00BB010A89828A83E0F5F0A3E022500687C9
:10070C00F009E71922BBFE07E3F5F009E31922898A
:0B071C00828A83E493F5F074019322BD
:10072700BB010789828A830206E6500B09C5F027B9
:10073700F7C5F01937F722BBFE0D09F8E325F0F3EB
:10074700C5F019E338F322F889828A837401932567
:08075700F0C5F0F8E49338222C
:10075F00BB010A89828A83F0E5F0A3F0225006F7E5
:0F076F0009A7F01922BBFE06F3E5F009F31922E2
:10077E00BC000BBE0029EF8DF084FFADF022E4CC5F
:10078E00F875F008EF2FFFEE33FEEC33FCEE9DEC28
:10079E00984005FCEE9DFE0FD5F0E9E4CEFD22ED6E
:1007AE00F8F5F0EE8420D21CFEADF075F008EF2FB8
:1007BE00FFED33FD4007985006D5F0F222C398FDA9
:0507CE000FD5F0EA2246
:00000001FF
